:0A00000032C0FECFFDCFFCCFFBCFD6
:10000A00FACFF9CFF8CFF7CFF6CFF5CF53C0F3CF6A
:10001A00F2CFF1CFF0CFEFCFEECFEDCF1027E8033D
:10002A0064000A0001000010000110000100000035
:10003A000000000000007E0CB69ECCDAFA0EFEDE4E
:10004A000100010002003800060006003A000A001A
:10005A006901400001007B014A000000F894EE2784
:10006A00ECBBF1E0FBBFEBBFE5BF8DE0A2E0BB2735
:10007A00ED938A95E9F780E094E0A0E6ED93019785
:10008A00E9F7ECE4F0E085919591009761F0A5918C
:10009A00B59105901590BF01F00105900D92019759
:1000AA00E1F7FB01F0CFEFE5EDBFE4E0EEBFC0E61C
:1000BA00D1E04AC0AA93EA93FA93EFB7EA93BDD282
:1000CA001BB10CB1E12FEC71D1F4E0918701EF5F24
:1000DA00E093870135D20083A0918701A83019F4F3
:1000EA00E0E0E0938701A0918901AF5FA0938901C5
:1000FA00A83029F4E0E0E0938901689420F8099196
:10010A001991E991EFBFF991E991A99118951A937B
:10011A00E0918901E030E1F3E0918801EF5FE0933B
:10012A0088010ED21081A0918801A83019F4E0E06C
:10013A00E0938801F894E0918901E150E093890104
:10014A007894E12F19910895CAD19FD0A0917B018B
:10015A00A13009F066C0E0916201E03009F05EC0AA
:10016A00A0916101A13039F4E1E0E0937701E0E088
:10017A00E093790153C0A0916101A23099F4E0E0C3
:10018A00E0937701A0916301A13029F4E1E0E093C3
:10019A007801E0E004C0E0E0E0937801E1E0E09378
:1001AA0079013CC0A0916101A330C1F5E0E0E09380
:1001BA007701A0917801A13009F401C0E1E0E09350
:1001CA007901A0916301A13011F4E1E001C0E0E0FE
:1001DA00E0937D01E0916401E03011F4E1E001C0B7
:1001EA00E0E0E0937E01E0916701E03021F0809049
:1001FA006701992402C088249924F0916501E0E0FE
:10020A002F01D0906601ED2DF0E0E429F5293F0198
:10021A00EFE0F7E2E615F70508F43F01E0E0E093C6
:10022A007B01A0917701A13009F48FD1A0917801C7
:10023A00A13019F5F50131965F01E0917C01E030BA
:10024A0069F4D30167D0E0EAFFE0EA15FB0529F477
:10025A00AA24BB24E1E0E0937C010FC0A0917C01B9
:10026A00A13059F472D1E8E9FAE3EA15FB0529F459
:10027A00AA24BB24E0E0E0937C01A0917901A1309B
:10028A0011F4D30147D061CFFFCFE0918901E0306B
:10029A0009F43FC03CDFCE2EAC2DE0EF5BD1E0E0AD
:1002AA00A7D1E02111F05BD134C0A0917A01E0E03E
:1002BA00A9D10E2EE8E0A1D1E02111F050D129C038
:1002CA00AC2DEDE047D1E8E093D1E02169F0E0916F
:1002DA007A01F0E0E05AFE4FC082E0E0E0937A0152
:1002EA00E1E0E0937B0115C0E0E0E0937A01E0935E
:1002FA006001E0936101E0936201E0936301E0939E
:10030A006401E0936501E0936601E0936701E0937D
:10031A0068010895BA93AA9324972CD178D1E093CF
:10032A00730128D187D1DF01E4E6F0E070D1E093D0
:10033A007401AC81BD81E4E6F0E07CD1DF01EAE042
:10034A00F0E065D1E0937501AC81BD81EAE0F0E0AF
:10035A0071D1E0937601E0E0E5BBE2BBA0917E01BA
:10036A00A13009F07CC00BD10ED1E030B1F507D134
:10037A00309721F404D10BD1E0E02DC0E130A0E0A8
:10038A00FA0779F4FCD0319702D1EC91E03021F4EC
:10039A00F6D0FDD0E0E003C0F2D0F9D0E1E0EC9372
:1003AA001BC0E230A0E0FA0779F4E9D03197EFD028
:1003BA00EC91E03021F4E3D0EAD0E0E003C0DFD0F2
:1003CA00E6D0E1E0EC9308C0E330A0E0FA0721F4BC
:1003DA00D6D0DDD0E1E0EC9305C0E1E0E883E98323
:1003EA00EA83EB83A0917D01A13011F4D4D009F006
:1003FA0002C0E0E830C0C3D0CAD0EC91E03019F4B2
:10040A00E0E0E2BB2AC0082C092809F1C4D011F4A3
:10041A00C6D009F002C0C09A19C0C6D0A13011F4E2
:10042A00C6D009F002C0C09A11C0BED0A23011F4E1
:10043A00C3D009F002C0C09A09C0B6D0A33011F4E3
:10044A00C0D009F002C0C09A01C0C09801C0C098CB
:10045A0096D099D0BBD0E2BBBED0E5BB34C0082C45
:10046A00092809F198D011F49AD009F002C0C09A6B
:10047A0019C09AD0A13011F49AD009F002C0C09ADA
:10048A0011C092D0A23011F497D009F002C0C09ADC
:10049A0009C08AD0A33011F494D009F002C0C09ADE
:1004AA0001C0C09801C0C098A0917D01A13011F48B
:1004BA0072D009F002C0E0E803C061D064D086D0EF
:1004CA00E2BB89D0E5BB70D0A33011F4E0E003C0F1
:1004DA00E0918A01EF5FE0938A0126960895E1E0B0
:1004EA00E7BBE0E0E8BBEFE0E4BBE0E0E5BBEEEF52
:1004FA00E1BBE0E0E2BBE3BFE2BFEFBDEEBDEDBDB5
:10050A00ECBDE7BDE6BDEBBDEABDE9BDE8BDE2BDB8
:10051A00E5BDE4BDE3BDE9BFE5BFE2E0EBB9E0E973
:10052A00EAB9E6E8E0BDE0E0E0BDE0E1E9B9E0E82B
:10053A00E8B9E0E0E0BFE6B9EDB9E6BF789408951E
:10054A00E150F0E0E158FE4F0895E0E0E2BBE5BB80
:10055A00C09808954DD00E2EA0917A010895E09189
:10056A007A01EF5FE0937A01E150F0E0E05AFE4F42
:10057A00C0820895AC81BD81E8EEF3E00895E09170
:10058A008A01F0E00895ED58FE4FE0810895DE01FA
:10059A00AE0FBF1F0895A0918A01A0300895E1E02F
:1005AA00F0E0E815F9050895A0918A010895E2E0BE
:1005BA00F0E0E815F9050895E4E0F0E0E815F9053A
:1005CA000895E8E0F0E0E815F9050895F0E0E75944
:1005DA00FE4FE0810895E0918A01A1E001D00895DB
:1005EA00EE230E2EEA2F19F0EE0F0A94E9F708957A
:1005FA00EA17E1E009F0EE270895AE17E1E008F006
:10060A00EE270895EA17E1E008F0EE27089500249E
:10061A00112490E1AA0FBB1F001C111C0E1A1F0AFD
:10062A0018F40E0E1F1E01C0A1609A9599F7FD01DC
:10063A00D0010895ECDFFD0108951A930A930895F5
:00000001FF
